

Microchip Technology PIC18 LITE Macro Assembler V1.37 build -260352376 
                                                                                               Wed Sep 14 21:29:41 2016

Microchip Technology Omniscient Code Generator v1.37 (Free mode) build 201603110536
     1                           	processor	18F4550
     2                           	fnconf	rparam,??,?,0
     3                           	opt	pw 120
     4                           	opt	lm
     5                           	psect	cinit,global,reloc=2,class=CODE,delta=1
     6                           	psect	cstackCOMRAM,global,class=COMRAM,space=1,delta=1
     7                           	psect	text0,global,reloc=2,class=CODE,delta=1
     8                           	psect	intsave_regs,global,class=BIGRAM,space=1,delta=1
     9                           	psect	rparam,global,class=COMRAM,space=1,delta=1
    10  0000                     _ADCON0	set	4034
    11  0000                     _ADCON0bits	set	4034
    12  0000                     _ADCON1	set	4033
    13  0000                     _ADCON2	set	4032
    14  0000                     _ADRESH	set	4036
    15  0000                     _ADRESL	set	4035
    16  0000                     _CCP1CON	set	4029
    17  0000                     _CCP1CONbits	set	4029
    18  0000                     _CCP2CON	set	4026
    19  0000                     _CCP2CONbits	set	4026
    20  0000                     _CCPR1L	set	4030
    21  0000                     _CCPR2L	set	4027
    22  0000                     _LATD	set	3980
    23  0000                     _PORTC	set	3970
    24  0000                     _PR2	set	4043
    25  0000                     _T2CON	set	4042
    26  0000                     _TRISA	set	3986
    27  0000                     _TRISC	set	3988
    28  0000                     _TRISD	set	3989
    29                           
    30                           ; #config settings
    31  0000                     
    32                           	psect	cinit
    33  007F76                     __pcinit:
    34                           	opt stack 0
    35  007F76                     start_initialization:
    36                           	opt stack 0
    37  007F76                     __initialization:
    38                           	opt stack 0
    39  007F76                     end_of_initialization:
    40                           	opt stack 0
    41  007F76                     __end_of__initialization:
    42                           	opt stack 0
    43  007F76  0100               	movlb	0
    44  007F78  EFBE  F03F         	goto	_main	;jump to C main() function
    45                           
    46                           	psect	cstackCOMRAM
    47  000001                     __pcstackCOMRAM:
    48                           	opt stack 0
    49  000001                     ??_main:
    50                           
    51                           ; 1 bytes @ 0x0
    52  000001                     	ds	2
    53                           
    54 ;;
    55 ;;Main: autosize = 0, tempsize = 2, incstack = 0, save=0
    56 ;;
    57 ;; *************** function _main *****************
    58 ;; Defined at:
    59 ;;		line 12 in file "main_ADC_PWM.c"
    60 ;; Parameters:    Size  Location     Type
    61 ;;		None
    62 ;; Auto vars:     Size  Location     Type
    63 ;;		None
    64 ;; Return value:  Size  Location     Type
    65 ;;                  1    wreg      void 
    66 ;; Registers used:
    67 ;;		wreg, status,2, status,0
    68 ;; Tracked objects:
    69 ;;		On entry : 0/0
    70 ;;		On exit  : 0/0
    71 ;;		Unchanged: 0/0
    72 ;; Data sizes:     COMRAM   BANK0   BANK1   BANK2   BANK3   BANK4   BANK5   BANK6   BANK7
    73 ;;      Params:         0       0       0       0       0       0       0       0       0
    74 ;;      Locals:         0       0       0       0       0       0       0       0       0
    75 ;;      Temps:          2       0       0       0       0       0       0       0       0
    76 ;;      Totals:         2       0       0       0       0       0       0       0       0
    77 ;;Total ram usage:        2 bytes
    78 ;; This function calls:
    79 ;;		Nothing
    80 ;; This function is called by:
    81 ;;		Startup code after reset
    82 ;; This function uses a non-reentrant model
    83 ;;
    84                           
    85                           	psect	text0
    86  007F7C                     __ptext0:
    87                           	opt stack 0
    88  007F7C                     _main:
    89                           	opt stack 31
    90                           
    91                           ;main_ADC_PWM.c: 13: TRISA=0;
    92                           
    93                           ;incstack = 0
    94  007F7C  0E00               	movlw	0
    95  007F7E  6E92               	movwf	3986,c	;volatile
    96                           
    97                           ;main_ADC_PWM.c: 14: TRISD=0;
    98  007F80  0E00               	movlw	0
    99  007F82  6E95               	movwf	3989,c	;volatile
   100                           
   101                           ;main_ADC_PWM.c: 15: ADCON0=0x01;
   102  007F84  0E01               	movlw	1
   103  007F86  6EC2               	movwf	4034,c	;volatile
   104                           
   105                           ;main_ADC_PWM.c: 16: ADCON0bits.CHS=1;
   106  007F88  50C2               	movf	4034,w,c	;volatile
   107  007F8A  0BC3               	andlw	-61
   108  007F8C  0904               	iorlw	4
   109  007F8E  6EC2               	movwf	4034,c	;volatile
   110                           
   111                           ;main_ADC_PWM.c: 22: ADCON1=0x0D;
   112  007F90  0E0D               	movlw	13
   113  007F92  6EC1               	movwf	4033,c	;volatile
   114                           
   115                           ;main_ADC_PWM.c: 27: ADCON2=0x00;
   116  007F94  0E00               	movlw	0
   117  007F96  6EC0               	movwf	4032,c	;volatile
   118                           
   119                           ;main_ADC_PWM.c: 41: TRISC = 0;
   120  007F98  0E00               	movlw	0
   121  007F9A  6E94               	movwf	3988,c	;volatile
   122                           
   123                           ;main_ADC_PWM.c: 42: PORTC = 0;
   124  007F9C  0E00               	movlw	0
   125  007F9E  6E82               	movwf	3970,c	;volatile
   126                           
   127                           ;main_ADC_PWM.c: 46: PR2 = 0b11111111;
   128  007FA0  68CB               	setf	4043,c	;volatile
   129                           
   130                           ;main_ADC_PWM.c: 48: T2CON = 0b00000111;
   131  007FA2  0E07               	movlw	7
   132  007FA4  6ECA               	movwf	4042,c	;volatile
   133                           
   134                           ;main_ADC_PWM.c: 50: CCP1CON = 0b00111100;
   135  007FA6  0E3C               	movlw	60
   136  007FA8  6EBD               	movwf	4029,c	;volatile
   137                           
   138                           ;main_ADC_PWM.c: 56: CCP2CON = 0b00111100;
   139  007FAA  0E3C               	movlw	60
   140  007FAC  6EBA               	movwf	4026,c	;volatile
   141  007FAE                     l663:
   142                           
   143                           ;main_ADC_PWM.c: 58: ADCON0bits.GO=1;
   144  007FAE  82C2               	bsf	4034,1,c	;volatile
   145                           
   146                           ;main_ADC_PWM.c: 59: while(ADCON0bits.GO){
   147  007FB0  D024               	goto	l671
   148  007FB2                     l665:
   149                           
   150                           ;main_ADC_PWM.c: 60: LATD=(ADRESL>>6);
   151  007FB2  44C3               	rlncf	4035,w,c	;volatile
   152  007FB4  46E8               	rlncf	wreg,f,c
   153  007FB6  0B03               	andlw	3
   154  007FB8  6E8C               	movwf	3980,c	;volatile
   155                           
   156                           ;main_ADC_PWM.c: 61: CCPR1L=ADRESH;
   157  007FBA  CFC4 FFBE          	movff	4036,4030	;volatile
   158                           
   159                           ;main_ADC_PWM.c: 62: CCP1CONbits.DC1B=(ADRESL>>6);
   160  007FBE  CFC3 F001          	movff	4035,??_main	;volatile
   161  007FC2  0E06               	movlw	6
   162  007FC4  6E02               	movwf	(??_main+1)& (0+255),c
   163  007FC6                     u25:
   164  007FC6  90D8               	bcf	status,0,c
   165  007FC8  3201               	rrcf	??_main,f,c
   166  007FCA  2E02               	decfsz	(??_main+1)& (0+255),f,c
   167  007FCC  D7FC               	goto	u25
   168  007FCE  3A01               	swapf	??_main,f,c
   169  007FD0  50BD               	movf	4029,w,c	;volatile
   170  007FD2  1801               	xorwf	??_main,w,c
   171  007FD4  0BCF               	andlw	-49
   172  007FD6  1801               	xorwf	??_main,w,c
   173  007FD8  6EBD               	movwf	4029,c	;volatile
   174                           
   175                           ;main_ADC_PWM.c: 66: CCPR2L=ADRESH;
   176  007FDA  CFC4 FFBB          	movff	4036,4027	;volatile
   177                           
   178                           ;main_ADC_PWM.c: 67: CCP2CONbits.DC2B=(ADRESL>>6);
   179  007FDE  CFC3 F001          	movff	4035,??_main	;volatile
   180  007FE2  0E06               	movlw	6
   181  007FE4  6E02               	movwf	(??_main+1)& (0+255),c
   182  007FE6                     u35:
   183  007FE6  90D8               	bcf	status,0,c
   184  007FE8  3201               	rrcf	??_main,f,c
   185  007FEA  2E02               	decfsz	(??_main+1)& (0+255),f,c
   186  007FEC  D7FC               	goto	u35
   187  007FEE  3A01               	swapf	??_main,f,c
   188  007FF0  50BA               	movf	4026,w,c	;volatile
   189  007FF2  1801               	xorwf	??_main,w,c
   190  007FF4  0BCF               	andlw	-49
   191  007FF6  1801               	xorwf	??_main,w,c
   192  007FF8  6EBA               	movwf	4026,c	;volatile
   193  007FFA                     l671:
   194  007FFA  A2C2               	btfss	4034,1,c	;volatile
   195  007FFC  D7D8               	goto	l663
   196  007FFE  D7D9               	goto	l665
   197  008000                     __end_of_main:
   198                           	opt stack 0
   199  0000                     wreg	equ	0xFE8
   200                           status	equ	0xFD8
   201                           wreg	equ	0xFE8
   202                           status	equ	0xFD8
   203                           
   204                           	psect	rparam
   205  0000                     wreg	equ	0xFE8
   206                           status	equ	0xFD8


Data Sizes:
    Strings     0
    Constant    0
    Data        0
    BSS         0
    Persistent  0
    Stack       0

Auto Spaces:
    Space          Size  Autos    Used
    COMRAM           95      2       2
    BANK0           160      0       0
    BANK1           256      0       0
    BANK2           256      0       0
    BANK3           256      0       0
    BANK4           256      0       0
    BANK5           256      0       0
    BANK6           256      0       0
    BANK7           256      0       0

Pointer List with Targets:

    None.

Critical Paths under _main in COMRAM

    None.

Critical Paths under _main in BANK0

    None.

Critical Paths under _main in BANK1

    None.

Critical Paths under _main in BANK2

    None.

Critical Paths under _main in BANK3

    None.

Critical Paths under _main in BANK4

    None.

Critical Paths under _main in BANK5

    None.

Critical Paths under _main in BANK6

    None.

Critical Paths under _main in BANK7

    None.

Call Graph Tables:

 ---------------------------------------------------------------------------------
 (Depth) Function   	        Calls       Base Space   Used Autos Params    Refs
 ---------------------------------------------------------------------------------
 (0) _main                                                 2     2      0       0
                                              0 COMRAM     2     2      0
 ---------------------------------------------------------------------------------
 Estimated maximum stack depth 0
 ---------------------------------------------------------------------------------

 Call Graph Graphs:

 _main (ROOT)

 Address spaces:
Name               Size   Autos  Total    Cost      Usage
BITCOMRAM           5F      0       0       0        0.0%
EEDATA             100      0       0       0        0.0%
NULL                 0      0       0       0        0.0%
CODE                 0      0       0       0        0.0%
COMRAM              5F      2       2       1        2.1%
STACK                0      0       0       2        0.0%
DATA                 0      0       0       3        0.0%
BITBANK0            A0      0       0       4        0.0%
BANK0               A0      0       0       5        0.0%
BITBANK1           100      0       0       6        0.0%
BANK1              100      0       0       7        0.0%
BITBANK2           100      0       0       8        0.0%
BANK2              100      0       0       9        0.0%
BITBANK3           100      0       0      10        0.0%
BANK3              100      0       0      11        0.0%
BITBANK4           100      0       0      12        0.0%
BANK4              100      0       0      13        0.0%
BITBANK5           100      0       0      14        0.0%
BANK5              100      0       0      15        0.0%
BITBANK6           100      0       0      16        0.0%
BANK6              100      0       0      17        0.0%
BITBANK7           100      0       0      18        0.0%
BANK7              100      0       0      19        0.0%
ABS                  0      0       0      20        0.0%
BIGRAM             7FF      0       0      21        0.0%
BITSFR               0      0       0      40        0.0%
SFR                  0      0       0      40        0.0%


Microchip Technology PIC18 Macro Assembler V1.37 build -260352376 
Symbol Table                                                                                   Wed Sep 14 21:29:41 2016

                     u25 7FC6                       u35 7FE6              __CFG_BOR$ON 000000  
            __CFG_BORV$3 000000             __CFG_CP0$OFF 000000             __CFG_CP1$OFF 000000  
                    l671 7FFA                      l663 7FAE                      l665 7FB2  
           __CFG_CPB$OFF 000000                      _PR2 000FCB                      wreg 000FE8  
           __CFG_LVP$OFF 000000             __CFG_WDT$OFF 000000                     _LATD 000F8C  
                   _main 7F7C                     start 1000            __CFG_IESO$OFF 000000  
          __CFG_MCLRE$ON 000000             ___param_bank 000010            __CFG_PLLDIV$5 000000  
                  ?_main 0001                    _T2CON 000FCA                    _PORTC 000F82  
          __CFG_USBDIV$2 000000                    _TRISA 000F92                    _TRISC 000F94  
                  _TRISD 000F95            __CFG_PWRT$OFF 000000            __CFG_WRT0$OFF 000000  
          __CFG_WRT1$OFF 000000           __CFG_EBTR0$OFF 000000           __CFG_FCMEN$OFF 000000  
         __CFG_EBTR1$OFF 000000            __CFG_WRTB$OFF 000000            __CFG_WRTC$OFF 000000  
         __CFG_EBTRB$OFF 000000                    status 000FD8          __initialization 7F76  
           __end_of_main 8000                   ??_main 0001            __activetblptr 000000  
                 _ADCON0 000FC2                   _ADCON1 000FC1                   _ADCON2 000FC0  
                 _ADRESH 000FC4                   _ADRESL 000FC3                   _CCPR1L 000FBE  
                 _CCPR2L 000FBB           __CFG_VREGEN$ON 000000           __CFG_XINST$OFF 000000  
         __CFG_STVREN$ON 000000               __accesstop 0060  __end_of__initialization 7F76  
        __CFG_PBADEN$OFF 000000            ___rparam_used 000001           __pcstackCOMRAM 0001  
                _CCP1CON 000FBD                  _CCP2CON 000FBA                  __Hparam 0000  
                __Lparam 0000                  __pcinit 7F76                  __ramtop 0800  
                __ptext0 7F7C     end_of_initialization 7F76              _CCP1CONbits 000FBD  
            _CCP2CONbits 000FBA      start_initialization 7F76         __CFG_LPT1OSC$OFF 000000  
       __CFG_WDTPS$32768 000000               _ADCON0bits 000FC2                 __Hrparam 0000  
               __Lrparam 0000            __size_of_main 0084    __CFG_CPUDIV$OSC1_PLL2 000000  
     __CFG_FOSC$HSPLL_HS 000000  
